:1016000012C02CC02BC02AC029C028C027C026C0A9
:1016100025C024C023C022C021C020C01FC01EC0BE
:101620001DC01CC01BC011241FBECFE5D4E0DEBF0F
:10163000CDBF10E0A0E6B0E0E2EAFDE102C0059017
:101640000D92A036B107D9F713E0A0E6B0E001C0D3
:101650001D92AA33B107E1F7D7D2A1C3D1CF9C0124
:10166000E199FECF3FBB2EBBE09A8DB308959C015C
:10167000E199FECF3FBB2EBB6DBB0FB6F894E29A4B
:10168000E19A0FBE0895E0E0F0E009950895899A87
:10169000A29AB99A089580912E038F5F80932E03AA
:1016A00090911402992321F480FF04C0C19803C0D3
:1016B000913009F4C19A8A3068F010922E03992370
:1016C00011F010923903809139038A3018F48F5F3A
:1016D0008093390308959091600080912B039817AF
:1016E00010F00AC0A8955D9BFDCFE92FF0E0E05017
:1016F000FE4F80818CB901C0AA989F5F90936000D3
:1017000008953CB180912A03882309F050C008B69F
:1017100000FE06C080911902813011F41092190266
:1017200080911902882371F43A32E9F588B7816013
:1017300088BF12BE109229033093280381E0809362
:1017400019020895813079F5909129039F5F909354
:1017500029039D3810F010921902E92FF0E0E959A1
:10176000FE4F308320912803230F209328039330CA
:1017700041F4832F8C5F8093FD018D3810F010921F
:1017800019028091FD01981771F4822F831B8093B9
:101790002803381741F480911902813021F4809395
:1017A0002A031092190288B7816088BF12BE08957B
:1017B000809103028B5F80932B03E0E0F2E090E0E6
:1017C0008150282F30E02E0F3F1F02C08191980FCB
:1017D000E217F307D9F7908381E080936000AA9A1B
:1017E00083E397E00197F1F701C0A8955D9BFDCFDA
:1017F000809100028CB90895EF92FF920F931F938E
:10180000CF93DF9320911A0230911B0240911C026A
:1018100050911D0220932F033093300340933103E6
:10182000509332038091150290911602A0911702F5
:10183000B0911802281739074A075B0789F1E09031
:101840003303F09034030091350310913603CAE15D
:10185000D2E020E030E0C90163E070E08CD24C813E
:10186000892B21F0842F8F5F821B03C0842F82502D
:10187000820FE80EF11C011D111DF901ED59FF4FFA
:1018800080832F5F3F4F219681E02030380719F782
:10189000E0923303F0923403009335031093360340
:1018A000DF91CF911F910F91FF90EF900895A89530
:1018B000E199FECF82E090E09FBB8EBB1DBA0FB6D0
:1018C000F894E29AE19A0FBE84E090E060E070E064
:1018D00047E35BE03BD286E090E060E070E047E306
:1018E0005BE034D288E090E060E070E047E35BE0EA
:1018F0002DD2E199FECF8AE090E09FBB8EBB8EEFA8
:101900008DBB0FB6F894E29AE19A0FBEA8950895A0
:10191000FF920F931F93F09068010091FF01809157
:101920006901801709F06CC110916B011130C9F584
:1019300080916C01813019F41093140202C010924E
:10194000140290911402913009F08CC08AE28093C5
:10195000000200930102F092020289E080930302E8
:1019600090930402909305028CE090E0909307021C
:101970008093060280E091E0909309028093080230
:1019800080912C0390912D0390930B0280930A0277
:10199000809137039091380390930D0280930C024D
:1019A0002EC11230C9F480911402813011F090E000
:1019B00059C020916C012093FF01E199FECF8AE08C
:1019C00090E09FBB8EBB2DBB0FB6F894E29AE19AD4
:1019D0000FBE1092140245C090E0133009F042C0CF
:1019E00080911402813009F03DC070916D0160E07A
:1019F00080916C01680F711D70932D0360932C030F
:101A000088E090E047E35BE0A1D1E199FECF1FBA07
:101A10001EBA8FEF8DBB0FB6F894E29AE19A0FBE13
:101A2000E199FECF81E090E09FBB8EBB8FEF8DBB35
:101A30000FB6F894E29AE19A0FBE10923303109217
:101A40003403109235031092360380E090E0A0E05A
:101A5000BFEF8093150290931602A0931702B093E4
:101A6000180291E080916B01853021F5809114027C
:101A7000813009F088C080916C0190916D01A09136
:101A80006E01B0916F0180931A0290931B02A09394
:101A90001C02B0931D0290E0E92FF0E0DF01A9598C
:101AA000BE4F1B968C91E65EFD4F84839F5F9038FE
:101AB00099F768C0863009F066C0809114028130C1
:101AC00009F061C090E0E92FF0E0DF01A959BE4FB5
:101AD0001B968C91E256FD4F80839F5F903899F75B
:101AE0008BDE20912F0330913003409131035091D0
:101AF000320320308BE0380780E0480780E0580749
:101B000010F090E040C08091150290911602A091D3
:101B10001702B091180282179307A407B50711F1B5
:101B2000CA01B90140E0F0D160912F0370913003F8
:101B3000809131039091320340E4E6D160912F030C
:101B400070913003809131039091320340E8DCD1F1
:101B500060912F0370913003809131039091320393
:101B600040ECD2D180912F0390913003A0913103AA
:101B7000B09132038093150290931602A09317023E
:101B8000B093180291E080916B01893039F5809112
:101B90001402813019F520916C0130916D01409152
:101BA0006E0150916F018091330390913403A091A5
:101BB0003503B0913603281739074A075B0711F040
:101BC00090E00CC0E199FECF1FBA1EBA81E08DBB38
:101BD0000FB6F894E29AE19A0FBE91E08AE2809300
:101BE000000200930102F092020283E0809303025C
:101BF00084E6809304021093050290930602D8DDD8
:101C00001F910F91FF9008951F93A8952FE088E1F1
:101C100090E00FB6F894A89581BD0FBE21BD10BC11
:101C200087E189B988E18AB9899AA29AB99AE19932
:101C3000FECF82E090E09FBB8EBBE09A8DB38F3FDA
:101C400009F435DE84E090E06FE27BE069D09093A8
:101C500038038093370386E090E06FE27BE060D04A
:101C6000909362008093610088E090E06FE27BE0F7
:101C700057D090932D0380932C03E199FECF8AE0F7
:101C800090E09FBB8EBBE09A8DB38093FF0184E010
:101C900083BF8BE08EBD80E09DE29BBD8ABD18E0D6
:101CA000A89508B604FE04C088B7806188BFF3DC3D
:101CB0005F9927DD5E9B16C05E9A909160008091CF
:101CC0002B03981710F00AC0A8955D9BFDCFE92F54
:101CD000F0E0E050FE4F80818CB901C0AA989F5F70
:101CE0009093600080912A03882319F011DE1092EE
:101CF0002A03809139038450843090F6109339037D
:101D00008CB390E0FC01E270F07081FDF9CF1FBA56
:101D10001EBAE09A8DB3813009F0C2CF0995C0CFC9
:101D2000DF92EF92FF920F931F937B018C01FB01D7
:101D30000995D82EC8010196F7010995982F8D2D88
:101D40001F910F91FF90EF90DF900895DF92EF9237
:101D5000FF920F931F93D72E7A018C01FA010995F8
:101D6000C80101966D2DF70109951F910F91FF9004
:101D7000EF90DF900895AA1BBB1B51E107C0AA1F7B
:101D8000BB1FA617B70710F0A61BB70B881F991F1C
:101D90005A95A9F780959095BC01CD010895F894C6
:021DA000FFCF73
:101F0000E0E0FBE009950895EF92FF920F931F9395
:101F1000CF93DF93A8950FB7E199FECF50E0DA0198
:101F2000A60FB71F83E0FD0180935700E89507B621
:101F300000FCFDCF83E6E82E80E0F82EE40EF51ECF
:101F4000BD0111E04D555F4FE701398120E08881E7
:101F5000F901E80FF11DCF01FB010C0110935700AF
:101F6000E895112482E090E0E80EF91E6E5F7F4F45
:101F7000E416F50649F785E0FD0180935700E895E2
:101F800007B600FCFDCF81E180935700E8950FBFB5
:0E1F9000DF91CF911F910F91FF90EF90089578
:0400000300001600E3
:00000001FF
